:020000040800F2
:10000000A006002005010008290100082B010008B6
:100010002D0100082F010008310100080000000038
:100020000000000000000000000000003301000894
:10003000350100080000000037010008F90400083D
:100040003B0100083B0100083B0100083B010008A0
:100050003B0100083B0100083B0100083B01000890
:100060003B0100083B0100083B0100083B01000880
:100070003B0100083B0100083B0100083B01000870
:100080003B0100083B0100083B0100083B01000860
:100090003B0100083B0100083B0100083B01000850
:1000A0003B010008490600083B0100083D05000827
:1000B00061060008710700089D0800083B01000860
:1000C0003B0100083B0100083B0100083B01000820
:1000D0003B0100083B0100083B0100083B01000810
:1000E0003B0100083B0100083B010008DFF810D08D
:1000F00000F02EF800480047110B0008AFF3008015
:10010000A00600200D488047DFF83400016841F464
:10011000E0210160BFF34F8FDFF82800DFF82810DF
:1001200001600A4800477047FEE7FEE7FEE7FEE78A
:10013000FEE7FEE7FEE7FEE7FEE7FEE72701000831
:1001400024ED00E00CED00E00003FA05ED000008EE
:10015000064C074D06E0E06840F0010394E8070014
:1001600098471034AC42F6D3FFF7C4FF080C0008E0
:10017000280C000870B5194C8320206000256560AC
:10018000A56017486060012000F048F861680843E6
:10019000606014490D60086840F002000860206843
:1001A00040F48030206020688003FCD5206840F057
:1001B0008070206020688001FCD5606820F003001A
:1001C0006060606840F002006060606840F4800039
:1001D0006060086840F01000086070BD00100240C8
:1001E00000841D000020024000487047001BB7003B
:1001F0000048704700A24A040549064A884202D0D6
:100200000549884201D110467047104670470000EA
:10021000002C014000A24A0400340140012804D00F
:10022000B0F5807F03DD012102E000202CE00021F9
:10023000802801DD012200E000220A44402801DD7F
:10024000012100E000210A44102801DD012100E025
:1002500000210A44082801DD012100E000210A44B0
:10026000042801DD012100E000210A44022801DD0B
:10027000012100E000211144012801DD012000E0FE
:1002800000200844C01D0001702800D100207047E4
:100290000F4A536943F001035361936943F40073B8
:1002A00093610C4A136843F480731360094B0A4A44
:1002B00044331361516100219160916800F00100A5
:1002C0004FF4565343EA40100143916070470000D9
:1002D00000100240082401400000024038B5836845
:1002E00043F480138360836823F46023836083680E
:1002F00001F0070443EA44438360124C002914D000
:10030000012914D0022914D0032914D00E4C052938
:1003100015D0FF21FF2907D0204600F081F800907A
:10032000BDF800004008208738BD0121F2E7022116
:10033000F0E70321EEE74FF080440221EAE70421D1
:10034000E8E70000002C0140000800402DE9F041E2
:1003500005460E462F4930488D4203D1816941F44C
:10036000007181612D498D4203D1816941F4806121
:1003700081610024FFF738FF0746FFF739FFB0FB24
:10038000F7F27000B0FBF2F0032801D8032120E05F
:100390000F2802D801240F211BE01B2802D80224B9
:1003A0001B2116E0392802D80324392111E05328F3
:1003B00002D8042453210CE06F2802D805246F21B1
:1003C00007E08F2802D806248F2102E0072440F29C
:1003D000DF1144EAC40040EA841040EA442040EAC5
:1003E000043040EAC43040EA844040EA4450E860C7
:1003F00040EA046040EAC4602861E86A20F47000C2
:10040000E862193151434808A96841F00101A96027
:10041000BDE8F081002401400010024000280140A6
:100420002DE9F0410D4604461146204600F0CCFA75
:10043000032707230626681E4FF0040C012D01D068
:10044000022D12D1218BC20007FA02F291432183BF
:10045000228B0CEBC00103FA01F822EA0802228386
:10046000228B06FA01F10A432283032D01D0042DC9
:100470000FD1A18BED1EEA009740B943A183A28B57
:100480000CEBC5018B409A43A283A28B8E40324372
:10049000A283228C012101EB800301FA03F39A432A
:1004A0002284228C800081400A43228406488442B0
:1004B00005D1B4F8440040F40040A4F84400A08DF5
:1004C000401C80B2BDE8F081002C0140426B22F05C
:1004D0001F024263426B0A434263704705498A68C0
:1004E00022F001028A60C860886840F001008860DC
:1004F000704700000000024001480068004700000B
:10050000B80000204FF0E0210A6942F004020A61BD
:100510006FF07F42904204D30A6922F004020A611C
:10052000C008486170470000024A1160024900019A
:1005300008707047B800002023ED00E070B53B491B
:1005400008883B4C82073B4DA4F12006A4F18000B3
:1005500018D50A8822F002020A800178012901D107
:10056000006A804728888107334802D400882080A9
:1005700003E000882188401A3080288880F002003B
:10058000288070BD0A88520718D50A8822F0040214
:100590000A804178012901D1406A80472888810674
:1005A000264802D40088608003E000886188401AF1
:1005B0007080288880F02000288070BD0A8812078B
:1005C00018D50A8822F008020A808178032901D10F
:1005D000806A804728888105194802D40088A08055
:1005E00003E00088A188401AB080288880F4007059
:1005F000288070BD0A88D206FBD50A8822F0100236
:100600000A80C178012901D1C06A80472888810405
:100610000C4802D40088E08003E00088E188401A9A
:10062000F080288880F40050288070BD102C014094
:1006300098000020202C0140342C0140382C01402F
:100640003C2C0140402C01400348018821F001016D
:100650000180024800690047102C0140180000206A
:1006600070B54FF08045288AC10740480AD0A98953
:10067000C90707D0298A21F0010129824069BDE814
:1006800070400047298A394C8A07384904F18804A8
:10069000A4F12006497916D52A8A22F002022A827C
:1006A000012901D1006B8047288C800702D4A88ED5
:1006B000208003E0A88E2188401A3080288C80F0AA
:1006C0000200288470BD2A8A520716D52A8A22F091
:1006D00004022A82012901D1406B8047288C8006C0
:1006E00002D4288F608003E0288F6188401A7080D0
:1006F000288C80F02000288470BD298A090717D52E
:10070000298A21F0080129828179012901D1806B90
:100710008047288C800502D4A88FA08003E0A88F92
:10072000A188401AB080288C80F40070288470BDA5
:10073000298AC906FBD5298A21F010012982C179AD
:10074000012901D1C06B8047288C800403D4B5F8FF
:100750004000E08004E0B5F84000E188401AF080F5
:10076000288C80F40050288470BD00001800002000
:1007700070B543490888C20742480BD00A1F128847
:10078000D20707D00A8822F001020A808069BDE8FA
:10079000704000470A883B4C3B4D04F1900492079F
:1007A000A4F1200618D50A8822F002020A80017AF4
:1007B000012901D1006C804728888107334802D481
:1007C0000088208003E000882188401A3080288833
:1007D00080F00200288070BD0A88520718D50A8868
:1007E00022F004020A80417A012901D1406C80473D
:1007F00028888106264802D40088608003E00088AB
:100800006188401A7080288880F02000288070BDA0
:100810000A88120718D50A8822F008020A80817A0D
:10082000012901D1806C804728888105194802D4AC
:100830000088A08003E00088A188401AB080288842
:1008400080F40070288070BD0A88D206FBD50A8823
:1008500022F010020A80C17A012901D1C06C8047C0
:10086000288881040C4802D40088E08003E00088D6
:10087000E188401AF080288880F40050288070BDFC
:100880001004004018000020200400403404004000
:10089000380400403C0400404004004070B5434927
:1008A0000888C20742480BD00A1F1288D20707D017
:1008B0000A8822F001020A80C069BDE87040004742
:1008C0000A883B4C3B4D04F198049207A4F12006A2
:1008D00018D50A8822F002020A80017B012901D181
:1008E000006D804728888107334802D40088208023
:1008F00003E000882188401A3080288880F00200B8
:10090000288070BD0A88520718D50A8822F0040290
:100910000A80417B012901D1406D804728888106EA
:10092000264802D40088608003E000886188401A6D
:100930007080288880F02000288070BD0A88120707
:1009400018D50A8822F008020A80817B012901D18A
:10095000806D804728888105194802D40088A080CE
:1009600003E00088A188401AB080288880F40070D5
:10097000288070BD0A88D206FBD50A8822F01002B2
:100980000A80C17B012901D1C06D8047288881047C
:100990000C4802D40088E08003E00088E188401A17
:1009A000F080288880F40050288070BD1008004036
:1009B000180000202008004034080040380800409B
:1009C0003C0800404008004070B504460D461949F7
:1009D00019488C4203D1816941F400618161B4F10D
:1009E000804F03D1C16941F00101C16113498C42BB
:1009F00003D1C16941F00201C16111498C4203D1A7
:100A0000C16941F00401C161FFF7F2FB06462046CF
:100A1000FFF7F2FBB6FBF0F0B5FBF0F0010C4A1C5F
:100A2000B0FBF2F02185401EA085A084112020801B
:100A300070BD0000002C0140001002400004004086
:100A400000080040044801688907FCD5416841F06E
:100A500002014160704700000000024002E008C847
:100A6000121F08C1002AFAD170477047002001E028
:100A700001C1121F002AFBD17047000010B54020B1
:100A8000FFF72CFDFFF7DEFF1D48806820F0010016
:100A90001B49886000242FE01A4800EB041080688E
:100AA00000BB184800EB04100168174800F07EF8FE
:100AB000144901EB0411C860124800EB0410C0682F
:100AC0001249884217DB0F4800EB04104068401CB5
:100AD0000C4901EB0411486064200A4901EB041140
:100AE000886008E0074800EB04108068401E054954
:100AF00001EB04118860641C042CCDDB10BD0000E8
:100B000000000240BC0000201C020020A3480B0093
:100B1000002014E000211F4A02EB001251601D4A20
:100B200002EB001291601B4A02EB0012D1601A49DD
:100B300051F82010174A02EB00121160401C0628E1
:100B4000E8DBFFF717FB1548FFF7DCFC1449012031
:100B5000FFF7EAFC48211348FFF7F8FB0221114890
:100B6000FFF7B4FCE12203210E48FFF7B7FB0E4963
:100B70000020FFF78DFB4FF0E020006940F00100FE
:100B80004FF0E02108610846006940F0020008616A
:100B900000BFFEE7BC00002000000020407E0500F2
:100BA0007D0A0008002401401C0200202DE9F04FBE
:100BB0004FF040024FF000034FF000044FF00005EB
:100BC0000F4FDFF84080934212D030F9139003FBAF
:100BD00001F606F03F0637F916A009FB0AFB5C4454
:100BE00038F916A009FB0AFB5D4403F10103EAE7AB
:100BF00084FB0410C5FB0510BDE8F00F00BD00002C
:100C0000280C0008A80C0008280D0008000000208F
:100C1000BC0000005C0A0008E40D0008BC000020D5
:100C2000E40500006C0A0008FF7F627F8A7D7D7A00
:100C30004276E3706E6AF262825A34511D47573C25
:100C4000FC302825F9188C0C000074F307E7D8DA7B
:100C500004CFA9C3E3B8CCAE7EA50E9D92951D8F9F
:100C6000BE89838576829E8000809E807682838581
:100C7000BE891D8F92950E9D7EA5CCAEE3B8A9C30B
:100C800004CFD8DA07E774F300008C0CF918282594
:100C9000FC30573C1D473451825AF2626E6AE37051
:100CA00042767D7A8A7D627F00008C0CF9182825B7
:100CB000FC30573C1D473451825AF2626E6AE37031
:100CC00042767D7A8A7D627FFF7F627F8A7D7D7A30
:100CD0004276E3706E6AF262825A34511D47573C85
:100CE000FC302825F9188C0C000074F307E7D8DADB
:100CF00004CFA9C3E3B8CCAE7EA50E9D92951D8FFF
:100D0000BE89838576829E8000809E8076828385E0
:100D1000BE891D8F92950E9D7EA5CCAEE3B8A9C36A
:100D200004CFD8DA07E774F31100000012000000C6
:100D3000130000001400000017000000180000005D
:100D400000000000000000000000000000000000A3
:100D50000000000000000000000000000000000093
:100D60000000000000000000000000000000000083
:100D70000000000000000000000000000000000073
:100D80000000000000000000000000000000000063
:100D90000000000000000000000000000000000053
:100DA0000000000000000000000000000000000043
:100DB0000000000000000000000000000000000033
:100DC0000000000000000000000000000000000023
:100DD0000000000000000000000000000000000013
:040DE000000000000F
:04000005080000ED02
:00000001FF
